:100000000C9434000C943E000C943E000C943E0082
:100010000C943E000C943E000C943E000C943E0068
:100020000C943E000C943E000C943E000C943E0058
:100030000C943E000C943E000C943E000C943E0048
:100040000C943E000C943E000C943E000C943E0038
:100050000C943E000C943E000C943E000C943E0028
:100060000C943E000C943E0011241FBECFEFD8E04C
:10007000DEBFCDBF0E9440000C9498000C9400009D
:10008000259A249890E050E040E22BE080E0215057
:1000900021F558131FC09F5F9430E8F094B1937F0F
:1000A00094B923E330E02150310941F594B19C60CB
:1000B00094B92A9A2B987FEF90E722E071509040F4
:1000C0002040E1F700C00000239829EB3BE02150DD
:1000D000310909F590E0582FD8CF33B13071832B17
:1000E00059F02D9A3FE768E371E03150604070406D
:1000F000E1F700C00000CBCF2D98F4CF95B1942745
:1001000095B99FEF56E761E0915050406040E1F7AC
:1001100000C00000C8CF95B1942795B95FEF66E79E
:1001200071E0515060407040E1F700C00000CFCF57
:04013000F894FFCF71
:00000001FF
